:100000000C942A000C943C000C943C000C943C0092
:100010000C943C000C943C000C943C000C943C0070
:100020000C943C000C9464000C943C000C943C0038
:100030000C943C000C943C000C943C000C943C0050
:100040000C943C000C943C000C943C000C943C0040
:100050000C943C0011241FBECFE5D4E0DEBFCDBF21
:1000600010E0A0E6B0E001C01D92A136B107E1F7B3
:100070000E943E000C9474000C9400008FEF8ABB29
:1000800087BB84BB81BB12BA85E083BF89B781601F
:1000900089BF789420E137E260E240E951E005C091
:1000A000CA010197F1F72150304021153105C1F700
:1000B00082B3862782BB80916000813011F4109258
:1000C000600020E137E2ECCF1F920F920FB60F9243
:1000D00011248F9381E080936000969A8F910F9006
:0C00E0000FBE0F901F901895F894FFCFF2
:00000001FF
